:030000000219FDE5
:03000B000200AA46
:03002B0002015C73
:03005B000202EBB3
:030073000202D8AE
:1000800002030406080C10182030406080040608A3
:100090000C10182030406080A0C00003070F1F0D17
:1000A0000D0403060D0503030202C2AFC0D0C0E079
:1000B000206214E5256009E473E525F4F58AD2622F
:1000C000D0E0D0D0D2AF3285268AC262E526F46075
:1000D0002F30682520720DD0E0D0D0C2B1C287C2C7
:1000E00081D2AF32C2B1C287C281206F0C206609B3
:1000F000740AD5E0FDE57B4280D0E0D0D0D2AF32AB
:10010000758A00C28DD26201F901B9306805206696
:1001100002D2B101B9306805206602D28701B93038
:100120006805206602D28101B9C28230680A206661
:10013000077408D5E0FDD2B101B9C28630680A2043
:1001400066077408D5E0FDD28701B9C28030680A1D
:100150002066077408D5E0FDD28101B9C2AFC2ADF7
:1001600053E6EFC0D0C0E0D2D3D2AFC2CEE52A6012
:1001700007207449152A21BD7800790020742EE5E6
:1001800080307E01F430E50278FF53DACF207E0321
:1001900043DA20307E0343DA10C2D8C271E58030E2
:1001A0007E01F430E50279FFC3E89970CB3061033A
:1001B000752A40207403752A40885CD27020740D23
:1001C000E52B6004152B21CD43DA01C2D820700243
:1001D00021E0A85C206102C27020740221DE882226
:1001E0007882B60403852224C3E52594404002D2D8
:1001F0006420CF0AD0E0D0D043E610D2AD32C2CFD7
:10020000053A7802E52A6005307402152AC3E55CD8
:1002100094014005755F00412A756000756900E52D
:100220005F2401F55F5003755FFF7982B7020D30DF
:100230006E1DC3E52294324016854C227982B703A5
:100240000E306E0BC3E52294324004798E8722C3B0
:10025000E5239522600840041523415E0523D8CA92
:100260000569E56970021569D56A63756A017805E3
:10027000C3E569956B4057C3E569956C50087801F3
:10028000756A03020292C3E569956D5005780175A0
:100290006A01C3E5629524401E7982B7040241C316
:1002A000206E14852462E569046003856B69756AB4
:1002B0000175233C0202CEE5622850057562FF41BC
:1002C000C3F562E5620470067560FF7569FFD0E0F2
:1002D000D0D043E610D2AD32C2AF53E67F7592FA6A
:1002E0007593FFC260759104D2AF32C2AF53E6EF8F
:1002F000C2ADC0D0C0E0C0F0D2D3D2AFA8FBA9FC41
:10030000C2D8307102615253DACF207E0343DA1033
:10031000307E0343DA20D271E580307E01F420E59F
:1003200002612988278928A13753DACF207E034329
:10033000DA20307E0343DA10C2D8C271307402A1D1
:10034000237800E580307E01F430E502A123885C4B
:10035000A10B53DACF207E0343DA20307E0343DA49
:1003600010C271206102812B53DACF207E0343DA61
:1003700010307E0343DA20C2D8D27188578958C31F
:10038000E89555F8E99556F97B007E087A00C3E8B0
:10039000948CE994005005755B00811D882178A23A
:1003A000E6A8216055C3E894C8E994005008E4D257
:1003B000E4FB7A0A61F8C3E89468E994015008E420
:1003C000D2E3FB7A0F61F8C3E894D0E994025008B5
:1003D000E4D2E2FB7A1E61F8C3E894A0E9940550E8
:1003E00008E4D2E1FB7A3C61F8C3E89498E9940808
:1003F0005008E4D2E0FB7A787E00C3E89559FCE926
:10040000955AFD30E70AECF42401FCEDF43400FDCC
:10041000755B00C3EC9AED9E5003755B01885989AA
:100420005A8557558558567802A10BC3E89527F889
:10043000E99528F9307C0281EF307B0281EF307A38
:100440000281E8207502814EE9FDE8FC816DE9C377
:1004500013F9E813F830790281E8E9C313F9E813D6
:10046000F830780281E8E9C313FDE813FC20612C21
:0F047000C3EC941CED940240028184ED701EC316
:10047F00EC94C850180529E52970021529C3E52900
:10048F00940A5002A123755C00D270A123E5296064
:10049F000215297400207F037896E624FAFEE434CF
:1004AF0000FFC3EC9EFCED9FFD50067800790081A4
:1004BF00EFC3EC94FFED9400400678FF790081EFD5
:1004CF00EC8572F0A4C5F0A2F733F879004003026F
:1004DF00050B78FF790002050BE9C313F9E813F850
:1004EF00307C0EE9600278FFC3E81338F8E434007B
:1004FF00F9C3E894FFE99400400278FF885CD2705A
:10050F00206102A123741FF4552F4BF52FC274EBFA
:10051F007002D274752A40307403752A0A30610252
:10052F00A13720740353DAFE207403752B20D0F00B
:10053F00D0E0D0D0D2AD43E6103279010205677911
:10054F0003020567790A020567791E020567796458
:10055F0002056779C80205677817E4D5E0FDD8FA78
:10056F00D9F6227A147B7802058E7A107B8C0205DD
:10057F008E7A0D7BB402058E7A0B7BC802058E79BD
:10058F0002E4C286D5E0FDD287D5E0FDC287D5E073
:10059F00FDD286D5E0FDE920E002D2B130E002D2F3
:1005AF0081E573D5E0FDE920E002C2B130E002C27F
:1005BF00817496D5E0FDD9C9EAF8D5E0FDD8FBDB0B
:1005CF00BEC28622C37C007D0075F00005F0EA33C1
:1005DF00FAEB33FB50F6EB13FBEA13FAC3E9FFE830
:1005EF00FEE89AF8E99BF95004EFF9EEF8B3EC3313
:1005FF00FCED33FDD5F0DFEDF9ECF822E889F08A58
:10060F0020D2D4F8A9F07B0030F70B7BFFF4240144
:10061F00F8E9F43400F9E88520F0A4ADF0F8E985A5
:10062F0020F0A4AFF0FEED2EF974003FFA7C04C366
:10063F00EA13FAE913F9E813F8DCF48BF030F70A50
:10064F00E8F42401F8E9F43400F9E889F0C2D4F8A9
:10065F00A9F0227882B60403020701C3E55C94195E
:10066F00401EE52D54067018206E3678057994E7F4
:10067F00146007780A1460027812C3E54198401F8E
:10068F00306E098564627569FF756A01852224E4FD
:10069F00F544F545F546F547F548C26E020701D218
:1006AF006E7994E7147013E523F43333F913F8E9F3
:1006BF00540104F9E854FE0206F5E714147014E52A
:1006CF0023F4333333F913F8E9540304F9E854FCF2
:1006DF000206FDE523F433333333F913F8E95407F6
:1006EF000404F9E854F8C39440F8E99400F98844F5
:1006FF00894522C3E54113F9E54013F8C3E5449852
:10070F00F8E54599F9500CC3E89480E994FF401639
:10071F00020739C3E8947FE9940050030207397840
:10072F007F7900020739788079FF8849894A22E565
:10073F00492546F8E54A3547F9854A20E43007014F
:10074F00F43548FA30E709C3EA94F0401502077709
:10075F00C3EA940F500302077778FF79FF7A0F02ED
:10076F000777780079007AF0C3E5249561500AC3C2
:10077F0074019524500B020795E54A20E70E0207F6
:10078F0095E54A30E706884689478A482278A5E6E4
:10079F00FAC3E54933F8E54A33F9D10BE930E70BF2
:1007AF00C3E89480E994FF4013E1CFC3E8947FE955
:1007BF0094005002E1CF787F7900E1CF788079FF04
:1007CF00E820E715C3E52398F84009C3E8940140F2
:1007DF00030207F678010207F6E8F424012523F84F
:1007EF0040030207F678FF884B2278A6E6FAA8475F
:1007FF00A94812060BE930E70CC3E89401E994FF0E
:10080F00401602082BC3E894FFE994005003020836
:10081F002B78FF790002082B780179FFE920E71583
:10082F00C3E54B98F84009C3E8940140030208520E
:10083F007801020852E8F42401254BF8400302081E
:10084F005278FF88242278FFC26420693D206A1203
:10085F00D264C3E541940A4009C3E5259440500290
:0D086F00C26479A1E76023E541601F74FFBA
:10087C008541F0848539F0306A0375F005A4F8C51C
:10088C00F0600278FFC3E895645002A86488632284
:10089C00C3E5409440E5419401E56350031401AD78
:1008AC00046002F563227883E6F520120F2975E8BF
:1008BC009012054975E890E5E820ECFBA8BDA9BEAF
:1008CC00120FCF756E55756F00C3740013FD745500
:1008DC00606613FC74552CFC74003DFDECFAEDFBCA
:1008EC00C3E89AE99B4014E56E2455F56EE56F3428
:1008FC0000F56FEA2CFAEB3DFB80E5AE6EAF6FC3F3
:10090C00E56F13F9E56E13F8C3E913F9E813F87AF8
:10091C0003C3E913F9E813F8DAF7AA201A7009757A
:10092C006E00756F000209441AEA6008EE28FEEFAB
:10093C0039FFDAF88E6E8F6F2275E890227883E695
:10094C00FFE5E820ECF7A8BDA9BE0570C3E57094DF
:10095C00084052757000E9FA79A0E76044EA700724
:10096C00E571601B02097FC3E895716010E5715059
:10097C0006600C1402098B0460F902098BE571F511
:10098C0071C394A8401B7561C0C394054013756175
:10099C0080C39405400B756140C394054003756199
:1009AC000075BB0622EFC39401601F7455601BC316
:1009BC00E894FFE994035012C3E8956EE9956F50E3
:1009CC0009E561600C15610209DDE561F460020561
:1009DC0061A861C3E524985002A824C3E89562403D
:1009EC000AA862E562F4600385626188258826E5C1
:1009FC0070B4070375BB1E22743279A787F0A4C5A7
:100A0C00F0A2F733F8C3E895614002A86188228808
:100A1C0024882588268864227540007541F022C2FE
:100A2C00AF75C820A8CCA9CDAA3A30CF010A75C899
:100A3C0024D2AFAB3BAC3C883B893CC3E89BF8E988
:100A4C009C206908F930670261374194AD3D8A3DBD
:100A5C00F9EA9DFA600478FF79FFAE3EAF3F8B3E1A
:100A6C008C3FA83BA93CC3E89EF8E99FF9C3E5413C
:100A7C0013FBE54013FAE82AF540E93BF541500633
:100A8C007540FF7541FF41DEAA40AB41AC40AD4122
:100A9C007E047F02C3EB940440021E1FC3EB940838
:100AAC0040021E1FC3ED13FDEC13FCDEF7C3EA9CE2
:100ABC00FAEB9DFBEF6009C3E913F9E813F8DFF7D4
:100ACC00EA28FAEB39FB8A408B4150067BFF8B40BE
:100ADC008B41C3EB94025002D2673069047F0361EF
:100AEC00097892E6FFC3E537948240110FC3E537CE
:100AFC0094A040010FC3EF940640027F057E02E5EF
:100B0C0041C4540FF9E541C454F0F8E540C4540F06
:100B1C0028F8C3E89EFAE99400FB4009C3EA940262
:100B2C00EB940050047A02E4FB6183AA40AB41EBE6
:100B3C00C4FEEAC4540F4EFCC3EA9CFAEB9400FBCF
:100B4C00C3E813C313F8EA28FAEB3400FB8A408B92
:100B5C0041C3EB94024002C2677802EBC4FE7B00F7
:100B6C00EAC4540F4EFAC3EA98FA4005C3940250F3
:100B7C00027A027892E6FF30600261838551928599
:100B8C005293D26043E680C3E49AF8E49BF9306751
:100B9C0002810FE8FAE9FBD3E913FDE813FC885155
:100BAC008952C3EF94036038EF20E00DE82CF8E98C
:100BBC003DF9ECFAEDFB020BD8E828F8E939F9C35A
:100BCC00E82402F8E93400F97AFE7BFFC3EF9403C2
:100BDC00400E8A538B54884D894E8C4F8D508143D7
:100BEC00885389548A4D8B4E8C4F8D5030691275B9
:100BFC0053F07554FF754FF07550FF7551F07552E9
:100C0C00FF8143E8FAD3E813FC8851C3EF940360E7
:100C1C0020EF20E007E82CF8ECFA812FE8282402DA
:100C2C00F87AFEC3EF940340088A53884D8C4F81A9
:100C3C004388538A4D8C4FE568C3335002646BF57F
:100C4C0068306002814D753402D26043E680E52D38
:100C5C0054066034A840A941C3E913F9E813F8C35A
:0F0C6C00E913F9E813F8306904E92440F9C2AF3D
:100C7B0053E67F759100C3E498F594E499F5957567
:100C8B009104D26043E680D2AF22D26575430075E2
:100C9B002000306C03752040020CB4D26575430004
:100CAB00752040306C037520007801790120672096
:100CBB00E52D54066002C2657914E541C31370013A
:100CCB0004F8C3941440027814306904781B791B20
:100CDB00206010E543600C306903D53404D26DA15C
:100CEB005691550543E59B5440B52002A140306910
:100CFB000908C3E89940011881DB20650A08C3E89D
:100D0B0099400281B481DBC265C2AF53E67F759116
:100D1B00003067127594007595FE759104D260438F
:100D2B00E680D2AF81B4AE40AF41C3E49EF594E40C
:100D3B009FF595A125C3E5339401500281B430652D
:100D4B000281B4D802A15481DBC26DC2AF53E67FDE
:100D5B00759100855394855495759104854D9285B5
:100D6B004E93D26043E680D2AFE52D540660082047
:100D7B006A020533020D92306D0D206C0A20650757
:100D8B001581158102161922780030640530650231
:100D9B007801E53775F007A4F9E5F028F5F0E9A23D
:100DAB00F013A2F113A2F213F537C3947850037525
:100DBB003778C3E53795384008D266C2B1C287C2CF
:100DCB0081306002A1CC854F92855093D26043E66F
:100DDB008022207D16C2AF754202C286D28230625B
:100DEB0002D281D2AF759F02020FCCC2AF75420205
:100DFB00C286D280306202D2B1D2AF759F02020F8F
:100E0B00CC307243207D20C2AF75420390013A75FE
:100E1B007B40C281C280306204D287C12AD286D283
:100E2B00AF759F03020FCCC2AF75420390013A75A9
:100E3B007B40C2B1C282306204D287C14AD286D211
:100E4B00AF759F01020FCC207D17C2AF7542039087
:100E5B000115C281306202D287D2AF759F03020F98
:100E6B00CCC2AF754203900115C2B1306202D2877A
:100E7B00D2AF759F01020FCC207D16C2AF75420415
:100E8B00C282D280306202D287D2AF759F01020F2D
:100E9B00CCC2AF754204C280D282306202D287D2FA
:100EAB00AF759F03020FCC307243207D20C2AF750C
:100EBB004205900129757B04C287C286306204D239
:100ECB00B1C1D0D282D2AF759F02020FCCC2AF7527
:100EDB00420590014B757B01C287C286306204D2FA
:100EEB0081C1F0D280D2AF759F02020FCC207D174B
:100EFB00C2AF75420590010BC287306202D2B1D2EC
:100F0B00AF759F02020FCCC2AF75420590011FC295
:100F1B00873062EBD281D2AF759F02020FCC207D5E
:100F2B0016C2AF754206C280D286306202D2B1D2EF
:100F3B00AF759F03020FCCC2AF754206C282D28639
:100F4B00306202D281D2AF759F01020FCC30724357
:100F5B00207D20C2AF75420190014B757B01C2B160
:100F6B00C282306204D281E176D280D2AF759F010A
:100F7B00020FCCC2AF754201900129757B04C2816F
:100F8B00C280306204D2B1E196D282D2AF759F0398
:100F9B00020FCC207D17C2AF75420190011FC2B169
:100FAB00306202D281D2AF759F01020FCCC2AF75F6
:100FBB00420190010BC281306202D2B1D2AF759F58
:100FCB0003C26622900109757B00C2B1C287C28140
:100FDB00C282C286C280C2622278807607087607F8
:100FEB000876010876040876FF0876FF087609086C
:100FFB007602087601087601788C7601087600086F
:10100B0076B40876FF0876FF0876FF087603087635
:10101B00FF0876010876FF0876250876D0087678E3
:10102B000876C80876040876FF087601087600086B
:10103B00767A08760A087601087601087600087633
:10104B00FF087600227887E6FFC272BF0302D272D6
:10105B007888C27DE630E102D27DC27E7889E630A7
:0F106B00E102D27EC3EF94026008758E01D2734A
:10107A00021082758E00C273227880E61490008076
:10108A009378A5F67881E6149000809378A6F6788E
:10109A0086E61490008D9378A7F6789FE6F870019B
:1010AA0008C3E8941140027811E82828F56B256BEB
:1010BA00256B28F56C256B2828F56D7886E6F539B9
:1010CA00C394025003753902789CE67538FFB4025E
:1010DA00037538A0B4030375388278A3E614900028
:1010EA009A93F566120FCF22227896E6FA7897E657
:1010FA00FB7888E6B40305C3EB940EFB307F047AD1
:10110A00007BFFC3EB9AFCC3948250027C82757207
:10111A00000572EC8572F0A4C3E5F0947D40F222DA
:10112A00D27F11F31205587A007B007C1012054E0B
:10113A00E55C2AFA74003BFBDCF37C04C3EB13FB8B
:10114A00EA13FADCF7FEC27F11F322E5EF20E60389
:10115A007520000520903DFFE520146006901FFFD2
:10116A001460009304600375EF1253D9BF7581C0F0
:10117A0043FF8012054975EF0243B203E5B3240227
:10118A0020E70DF521E5B120E0068521B343B10141
:10119A00120FCF75803875A4C775F1FF75D4DF7546
:1011AA0090FF75A50075F20075D50075A0FF75A6AC
:1011BA000075F30075D60075B0E475A71B75F4FFCA
:1011CA0075E241120FCFE4F8F6D8FD756801120FE7
:1011DA00E412167078988673753001C2AF120562F0
:1011EA001205721205581205791205581205801255
:1011FA00055812179312056212056212055DC2AFF5
:10120A0078FA79FA308507D9FBD8F7021C00115011
:10121A00118311F211F378988673120FCF75881023
:10122A0075890275C82475910475D84075A8227508
:10123A00B80275E690759B80759D0075D10E75BCD8
:10124A005875BB0675BA1F75E880120549D2AF12E8
:10125A0008B275360053DACF207E0343DA20307E97
:10126A000343DA1043DA01C2D8C271120562D261AD
:10127A007B037A0CE55B70077A0CDB030212081217
:10128A000558207003021208C270E55CC39402403C
:10129A00E1E52F541F855E5DF55EB55DD5DAD5C2F1
:1012AA006153DACF207E0343DA20307E0343DA101B
:1012BA00C2D8C27178A2E67008D274E52F54E0F55C
:1012CA002FC27575290012055D307409C3E529948A
:1012DA000A4002D27512054E78023074027800C3B1
:1012EA00E55C9840F0C2AF120572120572120572DF
:1012FA00D2AF120562754C0012054E788CE6C39483
:10130A000150030213D8E530C3940150030213D8E5
:10131A00207435C3E55C94FF50030213D8C2AF12A0
:10132A000587D2AF12055DC3E55C940150EFC2AFE9
:10133A00120572120553120572D2AF12055DC3E58A
:10134A005C94FF40E90218187F05D27F11F3120559
:10135A005DC2AFC27F11F3AE5CC3E55C947FD2AFCE
:10136A004076120549C2AF120587D2AFDFDC312AB7
:10137A00C3EE94057897F61205621216B212179BFD
:10138A007F0AD27F11F312055DC2AFC27F11F3AE9D
:10139A005CC3E55C947FD2AF50E6120549C2AF1236
:1013AA000572120553120572D2AFDFD6312AEE2426
:1013BA00037896F61205621216B21217CA12055D62
:1013CA0011F3C3E55C94FF5002611A021818C3E5D1
:1013DA005C954C4003855C4C12055D78017988E781
:1013EA00B403027805C3E55C9840026102C2AF12F9
:1013FA000587120587120587D2AF1205627530007C
:10140A00E4F531F5320531E531F4703F0532789A69
:10141A00E67819146012783214600D787D14600829
:10142A0078FA146003753200C3E53298401D120F32
:10143A00CF120549153275310078998673C2AF12F9
:10144A000587D2AF7898867312055D120553E52A8F
:10145A007005307402410878012074027806C3E5E9
:0E146A005C9840A112055DE52A70030212088D
:10147800C2AF120FCFE4F522F523F524F525F526A2
:10148800F567D2AF7885E6C333F565E4F544F545ED
:10149800F546F547F548F570F52CF52DF5377570D7
:1014A8000875BB1E120549120945E5E820ECFBA8A2
:1014B800BDA9BEE97001F8887112094975700875EF
:1014C800BB1E1150C2AF7561FF120A0485226185E7
:1014D8002262852263D2AF75220175240175250128
:1014E800752601856069756A017888E6B40307C2C4
:1014F8007D307602D27DD268D269753300120F2909
:10150800120F58120A24120A2B120A24120A2B123A
:101518000A24120CA6120662120D93120DDD120A8D
:101528002B120C95306E0312070220670312085520
:1015380030670312089C120D93120E0C120A2B121C
:101548000CA6306E0312073E120D93120E83120A78
:101558002B120C95306E0312079C120D93120EB2CB
:10156800120A2B120CA6306E031207F9120D9312F1
:101578000F29120A2B120945120C95120D93120FFE
:1015880058120949120A2B30692C856461856462F6
:10159800856069756A0179187A0CC3E53399400941
:1015A800C269D26A8A350215BEC3E55C940140035C
:1015B80002151A021621306A1D206C1AE5351470BE
:1015C80006C26AD26BA11AF535C3E55C94014003E3
:1015D80002151A021621753600C3E55F9401400909
:1015E800856462856069756A0178FA79A4E76002A2
:1015F8007803C3E55F985021307404E52A601A78AF
:10160800F0306C058564617820C3E541985002A1EB
:101618001A0536E55C6002C124753600C2AF120FA8
:10162800CF7887E6FE760211507887EEF6E4F52249
:10163800F523F524F525F526F565752C00752D009F
:10164800D2AF12055D120FCF78A4E66006D2B1D2F0
:1016580087D281307406E52A70024108788DE6C386
:101668009401400241DF810A901A0D78201216F485
:10167800E520B4A50CA31216F4E520B45A0302160B
:1016880092120FE41216B20216B1901A0378807BF8
:101698000A1216F4A308DBF9901A0F788C7B19123A
:1016A80016F4A308DBF9901A2822C2AF12173312D6
:1016B800170D901A00740E1216F9A374061216F973
:1016C800A374151216F9901A0378807B0A1216F87B
:1016D800A308DBF9901A0F788C7B191216F8A30867
:1016E800DBF9121746121724901A2822E493F622DF
:1016F800E6438F01538FFD75EF0275B7A575B7F1F6
:10170800F0538FFE22438F02438F0175EF0275B7A6
:10171800A575B7F1901A0DF0538FFC22901A0D742D
:10172800A5D1F9901A0E745AD1F9227A3079D07865
:1017380020901A40D1F4E520F709A3DAF7227A308D
:1017480079D0901A40E7D1F909A3DAF922AB74A845
:1017580075BB01027980BB02027981BB03027982E1
:10176800BB04027994BB05027983BB06027986BB68
:1017780007027992BB08027987BB0902799CBB0AE8
:10178800027988BB0B027989E8F7227C0512056289
:10179800DCFB22C2AF120572120579120580120510
:1017A80087120553120572120579120580120587F2
:1017B800120553120572120579120580120587D297
:1017C800AF22C2AF12058712058012057912057281
:1017D8001205531205871205801205791205721237
:1017E8000553120587120580120579120572D2AFCA
:1017F80022AE74AF75C2AF1205721205721205726D
:10180800120553DEF2120587120553DFF8D2AF2214
:1018180012179B121793121793757401757501753A
:1018280076001217F97C05AD5C120562C3ED955C74
:1018380070F5C3E55C9401400AC3E55C94FF40374A
:1018480002185C1217551216B212179BC2AF75EF29
:1018580012121793DCD10576C3E576940350028003
:0F186800C11217930575E5741490009F93F8084B
:10187700C3E57598500280A8121793121793057441
:10188700C3E574940C50028094120FE41216B2C28E
:07189700AF75EF1212179369
:0319FD000211557F
:101A00000E061507070104FFFF09020101A55A018F
:101A100000B4FFFFFF03FF01FF25D078C804FF01DA
:091A200000FF0A010100FF00FFB4
:101A4000235475726E696779343041232020202039
:101A500023424C48454C4923463331302320202033
:101A60002020202020202020202020202020202076
:101C0000C2AFC2D353D9BF7581C043B20343FF8073
:101C1000752438752503B1C975EF0275E24043F1AB
:101C20002053A4DF75D4FFD2857DFA780379E67C52
:101C300010752200752300901DD67B0675249875BB
:101C400025013085028142208508D8FBD9F9DCF7CF
:101C500081B4308508D8FBD9F9DCF781B4B189E4C7
:101C600093A3C39A6004DDC381B4DBDBB17B600264
:101C7000812B7B08E493FAA3B15CDBF87A30B15C8A
:101C8000752200752300B17BEAFCEBFDC3ED94FEE9
:101C9000400EB17B8A278B28ED30E0048A828B834B
:101CA000B17B7AC270D8C3ED94FE601350CEBD00F4
:101CB00025EC60097520007521FF0200008100A855
:101CC00027A9280809D804D90281D3B17FEA89AAB3
:101CD000F281C50D81A0C3ED94035049EDA2E092BD
:101CE000007AC5C3E5829400E583941C50902000DF
:101CF00010438F02438F0175B7A575B7F1F030001F
:101D00001FA827A9280809438F01538FFDD804D99C
:101D100002A12089AAE275B7A575B7F1F0A3A10DBC
:101D2000538FFC817C7AC1BD030CE493A3FAB140CC
:101D3000DCF8B138817C817EAA22AB23B15CEBFA5E
:101D4000EA6222752608C3E52313F523E52213F57D
:101D50002250066323A0632201D526EAB1C9B1C986
:101D600075260AEAF4200102D285300102C285B14B
:101D7000C9C3134002C201D526EB22B17FEAFB2082
:101D80008502A17F308502A184752608AE24AF2587
:101D9000C3EF13FFEE13FEB1CDB1C9C3EA13308513
:101DA000024480FA30E703632201C3E52313F523DD
:101DB000E52213F52250066323A0632201D526D91C
:101DC000E52265236523F52222AE24AF250E0FDE22
:101DD000FEDFFCD20122424C48656C693437316326
:041DE000F3100601F5
:00000001FF
